:0200000480007A
:100000009710000093800000171100001301810277
:1000100083A10000130210009302F0001303F0010B
:10002000930300001304000133924100B392510086
:1000300033936100B3937100339481002320310026
:10004000232241002324510023266100232871002C
:10005000232A810097100000938000FB17110000F5
:100060001301C1FE03A40000930410001305F00067
:100070009305F0011306000093060001B3149400E9
:100080003315A400B315B4003316C400B316D4005E
:1000900023208100232291002324A1002326B100E4
:1000A0002328C100232AD10097100000938000F676
:1000B00017110000130101FB83A6000013071000B5
:1000C0009307F0001308F0019308000013090001E2
:1000D0003397E600B397F60033980601B3981601FC
:1000E000339926012320D1002322E1002324F100AB
:1000F0002326010123281101232A210117160000BC
:10010000130606F197160000938646F703290600AA
:1001100093091000130AF000930AF001130B00007A
:10012000930B0001B3193901331A4901B31A59016C
:10013000331B6901B31B790123A0260123A23601D9
:1001400023A4460123A6560123A8660123AA76010B
:1001500017160000130606EC97160000938686F328
:10016000832B0600130C1000930CF000130DF0010C
:10017000930D0000130E0001339C8B01B39C9B0177
:10018000339DAB01B39DBB01339ECB0123A0760110
:1001900023A2860123A4960123A6A60123A8B601C3
:1001A00023AAC601971C0000938C0CE7171D0000C2
:1001B000130DCDEF03AE0C00930D1000B31EBE0166
:1001C000339FBE01B31FBF01B390BF013391B00194
:1001D000B311B1012320CD012322DD012324ED0140
:1001E0002326FD0123281D00232A2D00232C3D005A
:1001F00097100000938080E2171100001301C1ECFA
:1002000083A20000930D10003390B201232001005F
:10021000971000009380C0E017110000130101EB5C
:1002200083A20000930D10003390B201B312B0010D
:10023000232001002322510097100000938080DECC
:1002400017110000130101E983A10000370200101B
:10025000130202FEB7020010938212FE3703001051
:100260001303F3FEB70300109383F3FF33924100AF
:10027000B392510033936100B39371002320410086
:10028000232251002324610023267100171500004A
:10029000130545DA971500009385C5E4370610F07D
:1002A0001306C6F26306B5028326C5002320D600D6
:1002B000832685002320D600832645002320D600F0
:1002C000832605002320D600130505016FF09FFD4E
:1002D000370510F0130505F223200500000000008B
:0402E000000000001A
:101000000000000001000000FFFFFFFFFFFFFF7F67
:101010000000008010EFCDAB7856341298BADCFE99
:101020002143658700000000000000000000000070
:10103000FFFFFFFFFFFFFFFFFFFFFFFFFFFFFFFFC0
:10104000FFFFFFFFFFFFFFFFFFFFFFFFFFFFFFFFB0
:10105000FFFFFFFFFFFFFFFFFFFFFFFFFFFFFFFFA0
:10106000FFFFFFFFFFFFFFFFFFFFFFFFFFFFFFFF90
:10107000FFFFFFFFFFFFFFFFFFFFFFFFFFFFFFFF80
:10108000FFFFFFFFFFFFFFFFFFFFFFFFFFFFFFFF70
:10109000FFFFFFFFFFFFFFFFFFFFFFFFFFFFFFFF60
:1010A000FFFFFFFFFFFFFFFFFFFFFFFFFFFFFFFF50
:1010B000FFFFFFFFFFFFFFFFFFFFFFFFFFFFFFFF40
:1010C000FFFFFFFFFFFFFFFFFFFFFFFFFFFFFFFF30
:1010D000FFFFFFFFFFFFFFFFFFFFFFFFFFFFFFFF20
:040000058000000077
:00000001FF
